:020000020000FC
:100000000C94AB000C94C8000C94C8000C94C8006D
:100010000C94C8000C9453040C94C8000C94C800B1
:100020000C94C8000C9402010C94C8000C94C800F5
:100030000C94C8000C94C8000C94C8000C94C80020
:100040000C94C8000C94C8000C94C8000C94C80010
:100050000C94C8006E616E00696E660000407A10F4
:10006000F35A00A0724E18090010A5D4E80000E869
:100070007648170000E40B54020000CA9A3B0000C7
:1000800000E1F505000080969800000040420F0056
:100090000000A08601000000102700000000E80317
:1000A000000000006400000000000A0000000000E2
:1000B0000100000000002C76D888DC674F0823DFA1
:1000C000C1DFAE59E1B1B796E5E3E453C63AE65174
:1000D000997696E8E6C28426EB898C9B62ED407C9B
:1000E0006FFCEFBC9C9F40F2BAA56FA5F490055A37
:1000F0002AF75C936B6CF9676DC11BFCE0E40D475C
:10010000FEF520E6B500D0ED902E0300943577057E
:100110000080841E080000204E0A000000C80C3336
:100120003333330F986E12831141EF8D2114893BC5
:10013000E65516CFFEE6DB18D1844B381BF77C1D45
:10014000901DA4BBE424203284725E228100C9F198
:1001500024ECA1E53D2711241FBECFE5D8E0DEBF8A
:10016000CDBF10E0A0E6B0E0E6E9F3E102C0059003
:100170000D92A236B107D9F710E0A2E6B0E001C0B7
:100180001D92AE39B107E1F70E9433010C94C90901
:100190000C9400000C94003E089520E030E05F9B3A
:1001A000FECF8CB1F901E459FF4F80832F5F3F4FA1
:1001B00029313105A1F75F9BFECF8CB18E3729F035
:1001C0005D9BFECF85E48CB908955D9BFECF8EE7E5
:1001D0008CB981E08093640008958150E5E8F0E0F7
:1001E000E80FF11D80818BBBAC9A85818BBBAB9AEC
:1001F00082858BBBAA9A87858BBBA99A84898BBB86
:10020000A89A08951F920F920FB60F9211242F9360
:100210003F938F939F93F89480916500909166002F
:100220002091620030916300019782179307B1F02B
:100230008091620090916300019690936300809397
:10024000620081E08093640078949F918F913F9148
:100250002F910F900FBE0F901F9018951092630072
:1002600010926200EECF0E9486049FEF9ABB85E059
:1002700087BBC09A94BB91BBC29A1BBA15BA12BA7B
:100280008EB588618EBD8FB583608FBD8EB583605E
:100290008EBD89B7846089BF80E090E49BBD8ABD34
:1002A00085B5836085BD85B5886485BD8AE583BDD8
:1002B00089B7806489BFE0E8F3E1E4918E2F90E094
:1002C0009093660080936500E1E8F3E1E49120916A
:1002D0006500309166009E2F80E0820F931F9093FF
:1002E0006600809365007894C09841E05CE465E422
:1002F0007EE75F9BFECF8CB18A3209F580916B005F
:100300008130B9F720E030E05F9BFECF8CB1F9017E
:10031000E459FF4F80832F5F3F4F29313105A1F70B
:100320005F9BFECF8CB18E3721F05D9BFECF6CB909
:10033000E0CF5D9BFECF7CB940936400DACF83327F
:1003400029F412BAC09A0C94003ED3CF8C3451F0E9
:100350008E3479F610926B00C29A89B7846089BF97
:10036000C098C7CFC09A40936B0089B78B7F89BF75
:1003700080E090E0FC01E459FF4F10820196893142
:100380009105C1F7409364005D9BFECF5CB9B1CF8E
:10039000F89480916400882309F4FFC080E090E025
:1003A000FC01EE0FFF1FEE0FFF1FE80FF91FEB57C9
:1003B000FF4F1082118212821382148201968530BF
:1003C000910571F780916200909163002AE130E01D
:1003D000829FF001839FF00D929FF00D1124E05059
:1003E000FC4EF0936800E093670020916900309123
:1003F0006A0080916B00813009F4F2C0849180938F
:1004000085003196849180938A00319684918093FF
:100410008F003196849180939400319684918093DB
:100420009900759684917997482F50E0CA010197F9
:10043000449708F0D2C04B30510508F402C280E561
:1004400094E1489F9001499F300D589F300D112431
:10045000285538493BBD2ABD80916B00813009F495
:10046000DCC0359684918093860031968491809388
:100470008B00319684918093900031968491809383
:1004800095003196849180939A0070968491799723
:10049000482F50E0CA010197449708F476C128EC30
:1004A00032E33BBD2ABD80916B00813009F4D2C09C
:1004B0003A968491809387003196849180938C0042
:1004C0003196849180939100319684918093960027
:1004D0003196849180939B003B9684917997482F25
:1004E00050E0CA010197449708F42FC128EC32E389
:1004F0003BBD2ABD80916B00813009F4C8C03F9696
:100500008491809388003196849180938D003196F8
:1005100084918093920031968491809397003196D4
:10052000849180939C00369684917997482F50E06F
:10053000CA010197449708F4F8C028EC32E33BBDA8
:100540002ABD80916B00813009F4BEC074968491FD
:10055000809389003196849180938E0031968491A6
:100560008093930031968491809398003196849182
:1005700080939D0031968491482F50E0CA010197E5
:10058000449708F4F2C028EC32E33BBD2ABD309317
:100590006A00209369001092640012BA15BA1BBA5F
:1005A000979A80916000813009F4FFC080916000CB
:1005B000823009F412C180916000833009F425C1B2
:1005C00080916000843009F438C1809160008530EA
:1005D00009F493C097987894089528EC32E33ACFC1
:1005E00080916C008093850080916D0080938A00DB
:1005F00080916E0080938F0080916F0080939400B3
:10060000809170008093990088B394E0892788BB1B
:1006100080916B00813009F024CF8091710080932C
:1006200086008091720080938B008091730080938C
:100630009000809174008093950080917500809364
:100640009A0088B394E0892788BB80916B00813041
:1006500009F02ECF809176008093870080917700FB
:1006600080938C0080917800809391008091790034
:100670008093960080917A0080939B0088B394E0E9
:10068000892788BB80916B00813009F038CF809139
:100690007B008093880080917C0080938D00809106
:1006A0007D008093920080917E00809397008091DE
:1006B0007F0080939C0088B394E0892788BB809159
:1006C0006B00813009F042CF8091800080938900D7
:1006D0008091810080938E008091820080939300AE
:1006E00080918300809398008091840080939D0086
:1006F00088B394E0892788BB4ACF809189008BBB5F
:10070000AC9A80918E008BBBAB9A809193008BBB8F
:10071000AA9A809198008BBBA99A80919D008BBB6F
:10072000A89A969A9798789408954B30510508F4B2
:10073000B0C080E594E1489F9001499F300D589FDB
:10074000300D112428553849FACE4B30510508F4A4
:1007500096C080E594E1489F9001499F300D589FD5
:10076000300D112428553849C3CE4B30510508F4BB
:100770007CC080E594E1489F9001499F300D589FCF
:10078000300D11242855384900CF4B30510508F45D
:1007900062C080E594E1489F9001499F300D589FC9
:1007A000300D1124285538497CCE809185008BBBB3
:1007B000AC9A80918A008BBBAB9A80918F008BBBE7
:1007C000AA9A809194008BBBA99A809199008BBBC7
:1007D000A89A929A979878940895809186008BBBF6
:1007E000AC9A80918B008BBBAB9A809190008BBBB5
:1007F000AA9A809195008BBBA99A80919A008BBB95
:10080000A89A939A979878940895809187008BBBC3
:10081000AC9A80918C008BBBAB9A809191008BBB82
:10082000AA9A809196008BBBA99A80919B008BBB62
:10083000A89A949A9798789408950E94ED00959AB2
:10084000C9CE84E195E0489F9001499F300D589FA3
:10085000300D1124FFCD84E195E0489F9001499F20
:10086000300D589F300D11241CCE84E195E0489F37
:100870009001499F300D589F300D112486CE84E1A0
:1008800095E0489F9001499F300D589F300D1124ED
:100890002FCE84E195E0489F9001499F300D589FED
:1008A000300D11244CCE1F920F920FB60F921124CF
:1008B0002F933F934F935F936F937F938F939F9368
:1008C000AF93BF93EF93FF93F894809160008530CE
:1008D000C9F0809160008F5F809360000E94C80122
:1008E0007894FF91EF91BF91AF919F918F917F91FC
:1008F0006F915F914F913F912F910F900FBE0F908D
:100900001F90189581E080936000E8CF10BC8BE0C9
:1009100089B988E18AB986E880BD8CB15F99FDCF3D
:100920000895A1E1B0E0E7E9F4E00C9492093C01FC
:100930007F876E876A01FC0117821682838181FDA1
:1009400003C06FEF7FEF71C39E012F5F3F4F398B65
:10095000288BF3012381EE85FF8523FD859123FFFD
:100960008191FF87EE87882309F45CC3853251F4B7
:10097000EE85FF8523FD859123FF8191FF87EE871B
:10098000853229F490E0B3010E940809E2CF982F44
:1009900010E0882499241032B0F49B3269F09C3224
:1009A00028F4903251F0933271F40BC09D3239F03B
:1009B000903349F4116028C01260146025C018609B
:1009C00023C0106121C017FD2AC0892F80538A30AF
:1009D00078F416FF06C0FAE09F9E902C1124980E22
:1009E00013C03AE0839E802C1124880E10620CC044
:1009F0009E3221F416FD16C3106406C09C3611F415
:100A0000106802C0983659F4EE85FF8523FD959154
:100A100023FF9191FF87EE87992309F0BCCF892F9F
:100A20008554833020F4812F8061905E07C0892F28
:100A30008556833008F0A1C1812F8F7E86FD02C0CC
:100A400076E0972E6FE3F62EF822953619F4F0E44F
:100A5000FF2A07C0963619F420E8F22A02C0911046
:100A60009A94F7FE0BC03BE3391520F427E05CE3D2
:100A7000B52E0EC0B92CB39427E00AC047E0491543
:100A800028F427E0BB2447E0942E02C0292DBB2484
:100A9000C60104969D878C87F601608171818281F1
:100AA0009381AE014F5F5F4F0B2D0E941A086C01BE
:100AB0000981202E332400FF04C003FD02C01DE283
:100AC00009C0F1FE02C01BE205C0F2FC02C010E04A
:100AD00001C010E2C1018C709070892BB9F1112313
:100AE00011F483E001C084E0881510F088240AC066
:100AF000881AF3FC07C080E290E0B3010E94080965
:100B00008A94C9F7112329F0812F90E0B3010E9444
:100B1000080923FE03C004E510E00EC008E510E05C
:100B20000BC0E114F10409F0805290E0B3010E947F
:100B300008090F5F1F4F05C0EF2CFF24F0E1EF22E3
:100B4000FF24F8018491882361F714C1F7FE12C0D5
:100B5000BC0C24FE04C08A81813309F4BA941B14AE
:100B60001CF0BB24B3942DC0F8E0FB1550F538E021
:100B7000B32E27C0F6FC25C0892D90E08C159D056D
:100B80004CF02CEFC2162FEFD20624F030E8F32AF7
:100B900001C09A94992049F0E2E0F0E0EC0FFD1FCB
:100BA000E90DF11D80818033A1F3F7FE0AC0B92C55
:100BB000B394892D90E0C816D90614F0992401C089
:100BC0009C18F7FC03C025E030E009C01C141D048C
:100BD0001CF021E030E003C096012F5F3F4F11234E
:100BE00011F02F5F3F4F992029F0892D90E0019659
:100BF000280F391F882D90E02817390714F0882412
:100C000001C0821A4F2C5524C20189709070892B23
:100C100039F008C080E290E0B3010E9408098A948C
:100C20008820C1F7112329F0812F90E0B3010E94A1
:100C3000080943FE07C008C080E390E0B3010E94AA
:100C400008098A948820C1F7F7FE46C08601D7FEBE
:100C500002C000E010E076010894E11CF11CE01AEB
:100C6000F10A41E050E04C0F5D1FE40EF51E260135
:100C70004B185108892D90E0AA24BB24A81AB90A60
:100C80005FEF0F3F150729F48EE290E0B3010E9459
:100C90000809C016D10634F0401651061CF4F701BD
:100CA000808101C080E3015010400894E11CF11CD8
:100CB0000A151B052CF090E0B3010E940809E0CF53
:100CC0000C151D0539F49A81963318F4953311F4F7
:100CD00024FE81E390E04BC08A81813309F00F7ECE
:100CE00090E0B3010E9408099920A1F08EE290E003
:100CF000B3010E94080912E0E1E0F0E0EC0FFD1FF3
:100D0000E10FF11D1F5F808190E0B3010E9408098F
:100D10009A9491F744FC03C085E690E002C085E414
:100D200090E0B3010E940809D7FC05C0C114D104AA
:100D300041F404FF06C0D094C194D108D3948DE24D
:100D400001C08BE290E0B3010E94080980E305C076
:100D50008F5F26EF3FEFC20ED31E3AE0C316D104D9
:100D6000BCF790E0B3010E940809C601C096B30128
:100D70000E940809CC84DD8452C1933631F0933748
:100D800099F0933509F059C023C0F6018081898319
:100D90005E010894A11CB11C22E030E0C20ED31EFB
:100DA00021E0E22EF12C12C0F601A080B18016FDE8
:100DB00003C06FEF7FEF02C0692D70E022E030E0EA
:100DC000C20ED31EC5010E94FD087C011F7713C00F
:100DD000F601A080B18016FD03C06FEF7FEF02C067
:100DE000692D70E022E030E0C20ED31EC5010E94E2
:100DF000F2087C01106813FF07C01BC080E290E07E
:100E0000B3010E9408098A94882D90E0E816F9063B
:100E1000A8F30FC0F50117FD859117FF81915F01C0
:100E200090E0B3010E94080981108A940894E108B7
:100E3000F108E114F10471F7F2C0943611F099361B
:100E400089F517FF08C0F601208131814281538165
:100E500084E090E00AC0F601808191819C014427E2
:100E600037FD4095542F82E090E0C80ED91E9FE6D2
:100E7000F92EF12257FF09C05095409530952195E4
:100E80003F4F4F4F5F4F90E8F92ACA01B901AE01B9
:100E90004F5F5F4F2AE030E00E943409E82EE88976
:100EA000EE1A41C0953721F41F7E2AE030E01CC0C5
:100EB000197F9F3661F0903720F4983509F0B2C061
:100EC0000FC0903739F0983709F0ACC004C028E063
:100ED00030E00AC0106114FD146020E130E004C06D
:100EE00014FD166020E132E017FF08C0F6016081B2
:100EF00071818281938144E050E008C0F6018081D5
:100F00009181BC0180E090E042E050E0C40ED51E2B
:100F1000AE014F5F5F4F0E943409E82E5889E51AF1
:100F20008FE7F82EF122F6FE0BC08EEFF822E914BF
:100F300038F4F4FE07C0F2FC05C09FEEF92202C0AF
:100F40001E2D01C0192DF4FE0DC0FE01EE0DF11D88
:100F50008081803319F4E9EEFE2208C01F5FF2FEA3
:100F600005C003C08F2D867809F01F5F0F2DF3FC9D
:100F700014C0F0FE0FC0181510F09E2C0BC09E2C54
:100F8000980C911A182D06C080E290E0B3010E94DF
:100F900008091F5F1815C0F304C0181510F4811A52
:100FA00001C0882404FF0FC080E390E0B3010E94D9
:100FB000080902FF1DC001FD03C088E790E00EC0D4
:100FC00088E590E00BC0802F867891F001FF02C089
:100FD0008BE201C080E2F7FC8DE290E0B3010E9459
:100FE000080906C080E390E0B3010E9408099A94C2
:100FF000E914C0F3EA94E1E0F0E0EC0FFD1FEE0D20
:10100000F11D808190E0B3010E940809EE2091F764
:1010100006C080E290E0B3010E9408098A9488200B
:10102000C1F797CCF30166817781CB016196E2E14C
:101030000C94AE09283008F027E03327DA01990F25
:10104000311D87FD916000966105710539F43260AC
:101050002E5F3D9330E32A95E1F708959F3F30F0EE
:1010600080387105610509F03C5F3C5F3D9391302C
:1010700008F08068911DDF93CF931F930F93FF9229
:10108000EF92192F987F9695E92F96959695E90FEF
:10109000FF27EA54FF4F99273327EE24FF24A701A7
:1010A000E70105900894079428F4360FE71EF81E10
:1010B000491F511D660F771F881F991F0694A1F7BE
:1010C0000590079428F4E70EF81E491F561FC11D0E
:1010D000770F881F991F661F0694A1F70590079444
:1010E00028F4F80E491F561FC71FD11D880F991FDE
:1010F000661F771F0694A1F70590079420F4490F07
:10110000561FC71FD81F990F661F771F881F069489
:10111000A9F784911095177041F0D695C79557950A
:101120004795F794E7941A95C1F7ECE5F0E06894D9
:101130001590159135916591959105907FE2739584
:10114000E118F10A430B560BC90BD009C0F7E10CAB
:10115000F11E431F561FC91FD01D7EF4703311F4BA
:101160008A95E6CFE894015030F0080F0AF4002782
:10117000021708F4202F2395022F7A3328F079E301
:101180007D932A95E9F710C07D932A9589F60694F8
:1011900097956795379517951794E118F10A430BC2
:1011A000560BC90BD00998F023957E9173957A332D
:1011B00008F070E37C932013B8F77E9170617D9303
:1011C00030F0839571E37D9370E32A95E1F7112464
:1011D000EF90FF900F911F91CF91DF91992787FD9D
:1011E00090950895FC010590615070400110D8F76A
:1011F000809590958E0F9F1F0895FC01615070405F
:1012000001900110D8F7809590958E0F9F1F08953B
:101210000F931F93CF93DF938C01EB018B8181FFA1
:101220001BC082FF0DC02E813F818C819D812817BC
:10123000390764F4E881F9810193F983E88306C0F2
:10124000E885F985802F0995892B31F48E819F815E
:1012500001969F838E8302C00FEF1FEFC801DF91BD
:10126000CF911F910F910895FA01AA27283051F1CB
:10127000203181F1E8946F936E7F6E5F7F4F8F4FC7
:101280009F4FAF4FB1E03ED0B4E03CD0670F781F26
:10129000891F9A1FA11D680F791F8A1F911DA11D0B
:1012A0006A0F711D811D911DA11D20D009F4689444
:1012B0003F912AE0269F11243019305D3193DEF6EC
:1012C000CF010895462F4770405D4193B3E00FD0A2
:1012D000C9F7F6CF462F4F70405D4A3318F0495D8D
:1012E00031FD4052419302D0A9F7EACFB4E0A69570
:1012F0009795879577956795BA95C9F70097610592
:10130000710508959B01AC010A2E069457954795E7
:1013100037952795BA95C9F7620F731F841F951FDC
:10132000A01D08952F923F924F925F926F927F92ED
:101330008F929F92AF92BF92CF92DF92EF92FF92E5
:101340000F931F93CF93DF93CDB7DEB7CA1BDB0B91
:101350000FB6F894DEBF0FBECDBF09942A88398836
:1013600048885F846E847D848C849B84AA84B9843D
:10137000C884DF80EE80FD800C811B81AA81B98149
:10138000BE02FFFFFFFFFFFFFFFFFFFFFFFFFFFFAB
:10139000FFFFFFFFFFFFFFFFFFFFFFFFFFFFFFFF5D
:1013A000FFFFFFFFFFFFFFFFFFFFFFFFFFFFFFFF4D
:1013B000FFFFFFFFFFFFFFFFFFFFFFFFFFFFFFFF3D
:1013C000FFFFFFFFFFFFFFFFFFFFFFFFFFFFFFFF2D
:1013D000FFFFFFFFFFFFFFFFFFFFFFFFFFFFFFFF1D
:1013E000FFFFFFFFFFFFFFFFFFFFFFFFFFFFFFFF0D
:1013F000FFFFFFFFFFFFFFFFFFFFFFFFFFFFFFFFFD
:1014000000000000000000000000000000000000DC
:101410000000000000000000000A000000000000C2
:1014200000000000000000000000000000001F1F7E
:101430001F1F1F050000000000000000000000004A
:10144000000000000000001F1F1F1F1F00050000FC
:101450000000000000000000000000001F0000006D
:101460001F001F1F1F0000050000000000000000FB
:10147000001F0000001F0000001F00001F1F0000D1
:101480000005000000001F0000001F0000001F00FA
:1014900000001F0000001F00000000050000001FEA
:1014A0000000001F001F001F0000001F00000000C0
:1014B00000000000000500001F0000001F001F00CA
:1014C0001F0000001F0000000000000000000005D9
:1014D000001F0000001F001F00000000001F000090
:1014E0000000001F0000000000051F0000000000B9
:1014F0001F00000000001F00000000001F0000008F
:1015000000001F0500000000001F00000000001F79
:1015100000000000001F00000000001F1F05000069
:1015200000000000000000001F00000000001F007D
:10153000000000001F1F1F05000000000000000049
:10154000000000000000001F00000000001F1F1F1F
:101550001F05000000000000000000000000000067
:101560000000000000001F1F1F1F1F0500000000DB
:10157000000000000000000000000010101010101B
:101580000F0F0F0F0F05000000000000000000000B
:1015900010101010100808080808070707070705AB
:1015A00000000000001010101010080808080804BF
:1015B00004040404030303030305101010101008AF
:1015C00008080808040404040402020202020101DB
:1015D0000101010508080808081414141414020273
:1015E00002020201010101010000000000050404E3
:1015F0000404040A0A0A0A0A111111111100000058
:1016000000000000000000050202020202050505BC
:101610000505080808080810101010100000000048
:101620000005010101010102020202020404040496
:101630000408080808081010101010050000000029
:101640000001010101010202020202040404040477
:10165000181818181805000000000000000000000D
:10166000010101010102020202021C1C1C1C1C05DA
:101670000000000000000000000000000000000169
:10168000010101011E1E1E1E1E05000000000000BB
:1016900000000000000000000000000000001F1F0C
:1016A0001F1F1F05000000000000000000000000D8
:1016B0000000001F00000000001F1F1F1F0500008A
:1016C00000000000000000001F00000000001F00DC
:1016D000000000001F1F1F0500000000001F000089
:1016E0000000001F00000000001F00000000001F9D
:1016F0001F051F00000000001F00000000001F0069
:10170000000000001F00000000001F05001F000077
:10171000001F001F00000000001F00000000001F4D
:1017200000000000000500001F0000001F001F0057
:101730001F0000001F000000000000000000000566
:101740000000001F0000001F001F001F0000001FFE
:1017500000000000000000000005000000001F0065
:1017600000001F0000001F0000001F0000001F00FD
:10177000000000050000000000000000001F000045
:10178000001F0000001F00001F1F000000050000D8
:101790000000000000000000000000001F0000002A
:1017A0001F001F1F1F0000050000000000000000B8
:1017B00000000000000000000000001F1F1F1F1F8E
:1017C0000005000000000000000000000000000014
:1017D0000000000000001F1F1F1F1F050000000069
:1017E00000000000000000000000000101010101F4
:1017F0001E1E1E1E1E05000000000000000000004E
:10180000010101010102020202021C1C1C1C1C0538
:1018100000000000000101010101020202020204B5
:101820000404040418181818180501010101010224
:101830000202020204040404040808080808101044
:101840001010100502020202020505050505080830
:101850000808081010101010000000000005040413
:101860000404040A0A0A0A0A1111111111000000E5
:1018700000000000000000050808080808141414FF
:101880001414020202020201010101010000000021
:1018900000051010101010080808080804040404BB
:1018A0000402020202020101010101050000000020
:1018B000001010101010080808080804040404049C
:1018C0000303030303050000000000000000000004
:1018D0001010101010080808080807070707070568
:1018E00000000000000000000000000000000010E8
:1018F000101010100F0F0F0F0F0500000000000058
:1019000000000000000000000000000000001F1F99
:101910001F1F1F0500000000000000000000000065
:1019200000000000000000001F1F1F1F1F05000017
:1019300000000000000000000000000000000000A7
:10194000000000000000000A00000000000000008D
:101950000000000000000000000000000000000087
:101960001002000000000000000000000000000065
:101970000000000000100000000010020000000045
:101980000000000000000000000010000000001037
:101990000000000010020000000000000000001025
:1019A0000000000010000000001000000000000215
:1019B00000000000100000000010000000001000F7
:1019C00000000000000000000002000000101000F5
:1019D00000000010000000000000000000000000F7
:1019E00000000002000010101000000000000000C5
:1019F00000000000000000000000000000020010D5
:101A000010100000000000000000000000000000B6
:101A10000000000000000002101010000000000094
:101A200000000000000000000000000000000000B6
:101A30000002101000000010000000000000000074
:101A40000000000000000000000000021000000084
:101A50000010000000001000000000000000000066
:101A60000000000000020000000000100000000064
:101A70001000000000100000000000000000000244
:101A80000000000000000000000010000000001036
:101A90000000000010000000000200000000000034
:101AA0000000000000000000001000000000100016
:101AB0000000000200000000000000000000000024
:101AC0000000000000000000100000000002000004
:101AD0000000000000000000000000000000000006
:101AE00000000000000000020000000000000000F4
:101AF00000000000000000000000000008000000DE
:101B000000020000000000000000000000000000D3
:101B100000080000000008000000000200000000B3
:101B200000000000000008000000000800000000A5
:101B30000800000000020000000000080000000093
:101B40000800000000080000000000000000000283
:101B5000080000000008000000000800000000006D
:101B6000000000000000000000020808000000085B
:101B70000000000000000000000000000000000065
:101B8000000000020808080000000000000000003B
:101B9000000000000000000000000000000200083B
:101BA0000808000000000000000000000000000025
:101BB000000000000000000200000808080000000B
:101BC0000000000000000000000000000000000015
:101BD00000020000000808000000000800000000EB
:101BE00000000000000000000000000200000000F3
:101BF00008000000000800000000080000000000CD
:101C000000000000000200000000000000000008CA
:101C100000000000080000000008000000000002B2
:101C200000000000000000000000000000000800AC
:101C30000000000800000000080200000000000092
:101C4000000000000000000000000000000800008C
:101C5000000008020000000000000000000000007A
:101C6000000000000000000000000000080200006A
:101C70000000000000000000000000000000000064
:101C80000000000000000002000000000000000052
:101C90000000000000000000000000000000000044
:101CA000040200000000000000000000000000002E
:101CB000000000000004000000000402000000001A
:101CC000000000000000000000000400000000040C
:101CD00000000000040200000000000000000004FA
:101CE00000000000040000000004000000000002EA
:101CF00000000000040000000004000000000400D8
:101D000000000000000000000002000000040400C9
:101D100000000004000000000000000000000000BF
:101D200000000002000004040400000000000000A5
:101D3000000000000000000000000000000200049D
:101D4000040400000000000000000000000000008B
:101D50000000000000000002040404000000000075
:101D60000000000000000000000000000000000073
:101D70000002040400000004000000000000000055
:101D8000000000000000000000000002040000004D
:101D9000000400000000040000000000000000003B
:101DA000000000000002000000000004000000002D
:101DB0000400000000040000000000000000000219
:101DC000000000000000000000000400000000040B
:101DD00000000000040000000002000000000000FD
:101DE00000000000000000000004000000000400EB
:101DF00000000002000000000000000000000000E1
:101E000000000000000000000400000000020000CC
:101E100000000000000000000000000000000000C2
:101E200000000000000000020000000000000000B0
:101E300000000000000000000000000002000000A0
:101E40000002000000000000000000000000000090
:101E5000000200000000020000000002000000007C
:101E6000000000000000020000000002000000006E
:101E7000020000000002000000000002000000005C
:101E8000020000000002000000000000000000024C
:101E9000020000000002000000000200000000003C
:101EA000000000000000000000020202000000022A
:101EB0000000000000000000000000000000000022
:101EC000000000020202020000000000000000000A
:101ED00000000000000000000000000000020002FE
:101EE00002020000000000000000000000000000EE
:101EF00000000000000000020000020202000000DA
:101F000000000000000000000000000000000000D1
:101F100000020000000202000000000200000000B9
:101F200000000000000000000000000200000000AF
:101F3000020000000002000000000200000000009B
:101F4000000000000002000000000000000000028D
:101F5000000000000200000000020000000000027B
:101F6000000000000000000000000000000002006F
:101F7000000000020000000002020000000000005B
:101F8000000000000000000000000000000200004F
:101F9000000002020000000000000000000000003D
:101FA000000000000000000000000000020200002D
:101FB0000000000000000000000000000000000021
:101FC000000000000000000200000000000000000F
:101FD0000000000000000000000000000000000001
:101FE00001020000000000000000000000000000EE
:101FF00000000000000100000000010200000000DD
:1020000000000000000000000000010000000001CE
:1020100000000000010200000000000000000001BC
:1020200000000000010000000001000000000002AC
:10203000000000000100000000010000000001009D
:10204000000000000000000000020000000101008C
:10205000000000010000000000000000000000007F
:10206000000000020000010101000000000000006B
:10207000000000000000000000000000000200015D
:10208000010100000000000000000000000000004E
:10209000000000000000000201010100000000003B
:1020A0000000000000000000000000000000000030
:1020B000000201010000000100000000000000001B
:1020C000000000000000000000000002010000000D
:1020D00000010000000001000000000000000000FE
:1020E00000000000000200000000000100000000ED
:1020F00001000000000100000000000000000002DC
:1021000000000000000000000000010000000001CD
:1021100000000000010000000002000000000000BC
:1021200000000000000000000001000000000100AD
:10213000000000020000000000000000000000009D
:10214000000000000000000001000000000200008C
:10215000000000000000000000000000000000007F
:10216000000000000000020200000000000000006B
:10217000000000000000000000000002000000005D
:10218000020200000000000000000000000000004B
:102190000200000000020000000002020000000037
:1021A0000000000000020000000002000000000229
:1021B0000000000000020000000002000000000219
:1021C000000000000200000000000000000000020B
:1021D00000000002020000000002000000000000F9
:1021E00000000000000000000002000002020200E7
:1021F00000000000000000000000000000000000DF
:1022000000000002000202020000000000000000C6
:1022100000000000000000000000000000020202B8
:1022200002000000000000000000000000000000AC
:102230000000000000000002020200000002000096
:10224000000000000000000000000000000000008E
:102250000002020000000002000000000200000076
:10226000000000000000000000000002000000006C
:102270000002000000000200000000020000000058
:10228000000000000002000000000000000000004C
:102290000200000000020000000002000000000236
:1022A000000000000000000000000000000000022C
:1022B000000000000200000000020000000000001A
:1022C000000000000000000000000000000002000C
:1022D00000000002000000000000000000000000FC
:1022E00000000000000000000000000000020000EC
:1022F00000000000000000000000000000000000DE
:1023000000000000000004020000000000000000C7
:1023100000000000000000000000000400000000B9
:1023200004020000000000000000000000000000A7
:10233000040000000004000000000402000000008F
:102340000000000000040000000004000000000481
:102350000000000000020000000004000000000473
:102360000000000004000000000000000000000267
:102370000000000404000000000400000000000051
:10238000000000000000000000020000040404003F
:10239000000000000000000000000000000000003D
:1023A000000000020004040400000000000000001F
:1023B0000000000000000000000000000002040413
:1023C0000400000000000000000000000000000009
:1023D00000000000000000020404000000040000EF
:1023E00000000000000000000000000000000000ED
:1023F00000020400000000040000000004000000CF
:1024000000000000000000000000000200000000CA
:1024100000040000000004000000000400000000B0
:1024200000000000000200000000000000000000AA
:10243000040000000004000000000400000000028E
:102440000000000000000000000000000000000488
:102450000000000004000000000200000000000076
:102460000000000000000000000000000000040068
:10247000000000020000000000000000000000005A
:10248000000000000000000000000000000200004A
:10249000000000000000000000000000000000003C
:1024A0000000000000000802000000000000000022
:1024B0000000000000000000000000080000000014
:1024C0000802000000000000000000000000000002
:1024D00008000000000800000000080200000000E2
:1024E00000000000000800000000080000000008D4
:1024F00000000000000200000000080000000008CA
:1025000000000000080000000000000000000002C1
:1025100000000008080000000008000000000000A3
:102520000000000000000000000200000808080091
:10253000000000000000000000000000000000009B
:102540000000000200080808000000000000000071
:102550000000000000000000000000000002080869
:102560000800000000000000000000000000000063
:102570000000000000000002080800000008000041
:10258000000000000000000000000000000000004B
:102590000002080000000008000000000800000021
:1025A0000000000000000000000000020000000029
:1025B0000008000000000800000000080000000003
:1025C0000000000000020000000000000000000009
:1025D00008000000000800000000080000000002E1
:1025E00000000000000000000000000000000008E3
:1025F00000000000080000000002000000000000D1
:1026000000000000000000000000000000000800C2
:1026100000000002000000000000000000000000B8
:1026200000000000000000000000000000020000A8
:10263000000000000000000000000000000000009A
:102640000000000000000005000004000000000081
:10265000000000000000000000000000000000007A
:10266000000500000400000000040000000000005D
:102670000000000000000000000000050000040051
:102680000000000400000000040000000000000042
:10269000000000000005000004000000000400002D
:1026A000000004000000000400000000000000051D
:1026B000000004000000000400000000040000000E
:1026C00000040000000004000005000000000000FD
:1026D0000004000000000400000000040000000EE0
:1026E0000E0E0005000000000000000000000000C9
:1026F000040000000E0E0E00000E0E0E000500007D
:102700000000000000000000000E0A0E00000E0E87
:102710000E00000E0E0E00050000000000000E0A64
:102720000E00000E0A0E00000E0A0E00000E0E0E25
:102730000005000E0A0E00000E0A0E00000E0A0E22
:1027400000000E0A0E00000E0A0E00051F1F1B1FC0
:102750001F000E0A0E00000E0A0E00000E0A0E00E8
:102760000000000000051F1F1B1F1F1F1F1B1F1F36
:10277000000E0A0E0000000000000000000000052E
:102780001F1F1B1F1F1F1F1B0F1F1F1111111F00BA
:10279000000000000000000000051F1F1B1F1F1F7E
:1027A0001111111F1F1111111F1F1111111F0000F5
:1027B000000000051F1111111F1F1111111F1F1102
:1027C00011111F1F1111111F1F1111111F050000E1
:1027D0000000001F1111111F1F1111111F1F1111D6
:1027E000111F1F1F1B1F1F0500000000000000001D
:1027F00000001F1111111F1F1F1B1F1F1F1F1B1F59
:102800001F0500000000000000000000000E0A0E7E
:10281000001F1F1B1F1F1F1F1B1F1F050000000085
:1028200000000E0A0E00000E0A0E00000E0A0E0036
:102830001F1F1B1F1F05000E0A0E00000E0A0E00B0
:10284000000E0A0E00000E0A0E00000E0A0E000511
:102850000000040000000E0A0E00000E0A0E000028
:102860000E0A0E00000E0A0E000500000400000013
:1028700000040000000E0A0E00000E0A0E00000EFA
:102880000A0E000500000400000000040000000023
:10289000040000000E0A0E00000E0A0E00050000E3
:1028A0000400000000040000000004000000000418
:1028B0000000000E0A0E00050000040000000004E5
:1028C00000000000040000000004000000000400FC
:1028D00000050000000000000004000000000400EB
:1028E00000000004000000000400000500000000DB
:1028F00000000000000000000400000000040000D0
:1029000000000400000500000000000000000000BE
:1029100000000000000000040000000004000005AA
:1029200000000000000000000000000000000000A7
:10293000000000000000040000050000000000008E
:102940000000000000000000000000000000000087
:102950000000000500000000000000000000000072
:102960000000000000000000000A040A000500004A
:102970000000000000000000000000000000000453
:102980000000000A000A000500000000000000002E
:10299000000000000400000000000000000A000A1F
:1029A000000500000000000000040000000000001E
:1029B000000000000000000A000A000500000400FA
:1029C0000000000000000000000000000000000007
:1029D000000A000A000500040E04000000000000C8
:1029E00000000000000000000000000A000A0005CE
:1029F00000040A04000000000000000000000000C5
:102A000000000000000A000A000504001100040094
:102A10000000000000000000000000000000000AAC
:102A2000000A00050000000000040011000400007E
:102A30000000000000000000000A000A000500007D
:102A4000000000000000000004001100040000006D
:102A50000000000A000A000500000000000000005D
:102A6000000000000000000400110004000A000A39
:102A70000005000000000000000000000000000051
:102A8000000000000000040A110A04050000000014
:102A90000000000000000000000000000000000036
:102AA000000A000A0005000000000000000000000D
:102AB000000000000000020000000008000A0005FD
:102AC0000000000000000000000000020000000004
:102AD000000000000008000A0005000000000000DF
:102AE00002000000000000000000000000000008DC
:102AF000000A0005000200000000000000000000C5
:102B000000000000000000000008000A00050207A5
:102B100002000000000000000000000000000000B3
:102B200000000008000A0005020502000000000085
:102B30000000000000000000000000000008000A83
:102B4000000502010200000000000000000000007B
:102B50000000000000000008000A0005020100005B
:102B60000000000000000000000000000000000065
:102B70000008000A0005020000000000000000003C
:102B8000000000000000000000000008000A00052E
:102B90000000000000000000000000000000000035
:102BA000000000000008000A00050000000000000E
:102BB000000000000000000000000000020000080B
:102BC0000008000A000000000000000000000000F3
:102BD00000020000000000000008000800050000DE
:102BE00000000000000002000000000000000000E3
:102BF00000000008000800050000020702000000B5
:102C000000000000000000000000000000080008B4
:102C100000050000020502000000000000000000A6
:102C20000000000000000008000800050000020588
:102C30000000000000000000000000000000000094
:102C40000008000800050000020400000000000069
:102C5000000000000000000000000008000800055F
:102C60000000000400000000000000000000000060
:102C7000000000000008000800050000000000003F
:102C8000000000000000000000000000000000083C
:102C90000008000500000000000000000000000027
:102CA000000000000000080000080000000500000F
:102CB000000000000000000000000008000000000C
:102CC00000000008000000050000000000000000F7
:102CD00008000000000000000000000000080000E4
:102CE00000050000000800000000000000000000D7
:102CF0000000000000000008000000050000081CA3
:102D000008000000000000000000000000000000BB
:102D10000008000000050000081408000000000082
:102D20000000000000000000000000080000000596
:102D30000000081008000000000000000000000073
:102D4000000000000008000000050000001008005E
:102D5000000000000000000000000000000000086B
:102D60000000000500000000080000000000000056
:102D70000000000000000000000800000005000046
:102D80000000000000000000000000000000000043
:102D90000000000800000005000000000000000026
:102DA0000000000000000000080000000008000013
:102DB000000500000000000000000000000000000E
:102DC00000000800000000000000000500000000F6
:102DD00000000000000000080000000000000000EB
:102DE00000000000000500000000000008000000D6
:102DF00000000000000000000000000000000005CE
:102E000000080000000000000000000000000000BA
:102E100000000000000000000005081C0800000081
:102E200000000000000000000000000000000000A2
:102E30000000000508140800000000000000000069
:102E40000000000000000000000000000005081461
:102E50000000000000000000000000000000000072
:102E60000000000000000005081000000000000045
:102E70000000000000000000000000000000000052
:102E8000000500100000000000000000000000002D
:102E9000000000000000000000000005000000002D
:102EA0000000000000000000000000000000000022
:102EB000000000000005000000000000000000000D
:102EC00000000000000000000000000004000005F9
:102ED00000000000000000000000000000000000F2
:102EE00000040000000000000005000000000000D9
:102EF00000000000000004000000000000000000CE
:102F000000000005000000000000000400000000B8
:102F100000000000000000000000000000050000AC
:102F200004000000040E0400000004000000000083
:102F30000000000000000005000004000000040A7A
:102F40000400000004000000000000000000000079
:102F50000005000000000004001100040000000053
:102F6000000000000000000000000005000000005C
:102F70000000000000000400110004000000000038
:102F8000000000000005000000000000000000003C
:102F90000000000000040011000400000000000513
:102FA0000000000000000000000000000000000021
:102FB00000000000040011000405000000000000F3
:102FC0000000000000000000000000000000000001
:102FD000000000051010101010101010101010102C
:102FE00010101010101010101010101010051010EC
:102FF00010101010101010101010101010101010D1
:1030000010101010101008021010101010101010D6
:1030100010101010101010101010101010101010B0
:1030200004021010101010101010101010101010BA
:1030300010101010101010101010020210101010AC
:103040001010101010101010101010101010101080
:10305000101010100102101010101010101010108D
:10306000101010101010101010101010101100027D
:103070001010101010101010101010101010101050
:10308000101010101010111000021010101010105D
:10309000101010101010101010101010101010112F
:1030A000101000021010101010101010101010103E
:1030B000101010101010101011101010000210102D
:1030C0001010101010101010101010101010101000
:1030D000101011101000100210101010101010100D
:1030E00010101010101010101010101011101000EF
:1030F00008021010101010101010101010101010E6
:1031000010101010101011101000040210101010E8
:1031100010101010101010101010101010101010AF
:1031200011101000020210101010101010101010CA
:1031300010101010101010101010111010000102BB
:10314000101010101010101010101010101010107F
:10315000101010101110100100021010101010109B
:10316000101010101010101010101010101011105E
:10317000110000021010101010101010101010107C
:10318000101010101010101011111000000210106B
:10319000101010101010101010101010101010102F
:1031A000101011110010000210101010101010104B
:1031B000101010101010101010101010111100002D
:1031C000100210101010101010101010101010100D
:1031D0001010101010101111000008021010101023
:1031E00010101010101010101010101010101010DF
:1031F0001111000004021010101010101010101007
:1032000010101010101010101010111100000202F8
:1032100010101010101010101010101010101010AE
:1032200010101010111100000102101010101010D9
:10323000101010101010101010101010101011118C
:1032400000010002101010101010101010101010BB
:1032500010101010101010101111010000021010A9
:10326000101010101010101010101010101010105E
:103270001010110111000002101010101010101089
:10328000101010101010101010101010110101105B
:10329000000210101010101010101010101010104C
:1032A0001010101010101101010010021010101059
:1032B000101010101010101010101010101010100E
:1032C0001101010008021010101010101010101041
:1032D0001010101010101010101011010100040235
:1032E00010101010101010101010101010101010DE
:1032F0001010101011010100020210101010101017
:1033000010101010101010101010101010101101CB
:1033100001000102101010101010101010101010E9
:1033200010101010101010101101010100021010E7
:10333000101010101010101010101010101010108D
:1033400010100111010100021010101010101010C7
:103350001010101010101010101010100101110199
:10336000000210101010101010101010101010107B
:103370001010101010100101011100021010101097
:10338000101010101010101010101010101010103D
:103390000101010110021010101010101010101077
:1033A000101010101010101010100101010108026F
:1033B000101010101010101010101010101010100D
:1033C0001010101001010101040210101010101053
:1033D000101010101010101010101010101001010B
:1033E0000101020210101010101010101010101017
:1033F0001010101010101010010101010102101026
:1034000010101010101010101010101010101010BC
:10341000100801010101010210101010101010100D
:1034200010101010101010101010100401010101E4
:1034300001021010101010101010101010101010A9
:1034400010101010100201010101010210101010E3
:10345000101010101010101010101010101010017B
:1034600001010101010210101010101010101010B5
:1034700010101010101010101100010101010102B4
:10348000101010101010101010101010101010103C
:103490001011100001010101010210101010101094
:1034A0001010101010101010101011101000010149
:1034B0000101010210101010101010101010101047
:1034C0001010101110101000010101010102101064
:1034D00010101010101010101010101010111010EB
:1034E0000010010101010102101010101010101045
:1034F000101010101010101110100008010101011F
:1035000001021010101010101010101010101010D8
:10351000101110100004010101010102101010101F
:1035200010101010101010101010101110100002B8
:1035300001010101010210101010101010101010E4
:1035400010101010101110100001010101010102F2
:10355000101010101010101010101010101010116A
:1035600010100100010101010102101010101010D3
:103570001010101010101010101110110000010187
:103580000101010210101010101010101010101076
:1035900010101011111000000101010101021010A2
:1035A0001010101010101010101010101011110029
:1035B0001000010101010102101010101010101074
:1035C0001010101010101011110000100101010155
:1035D0000102101010101010101010101010101008
:1035E000101111000008010101010102101010105A
:1035F00010101010101010101010101111000004F5
:103600000101010101021010101010101010101013
:10361000101010101011110000020101010101022F
:103620001010101010101010101010101010101199
:103630001100000101010101010210101010101011
:1036400010101010101010101011110001000101C5
:1036500001010102101010101010101010101010A5
:1036600010101011110100000101010101021010E0
:103670001010101010101010101010101011011157
:1036800000000101010101021010101010101010B3
:103690001010101010101011010110000101010193
:1036A0000102101010101010101010101010101037
:1036B0001011010100100101010101021010101090
:1036C000101010101010101010101011010100082F
:1036D0000101010101021010101010101010101043
:1036E000101010101011010100040101010101026C
:1036F00010101010101010101010101010101011C9
:10370000010100020101010101021010101010104E
:103710001010101010101010101101010001010103
:1037200001010102101010101010101010101010D4
:10373000101010110101010001010101010210101E
:103740001010101010101010101010101001110196
:1037500001000101010101021010101010101010E1
:1037600010101010101010010111010001010101D1
:103770000102101010101010101010101010101066
:1037800010010101110001010101010210101010CE
:103790001010101010101010101010010101011065
:1037A0000101010101021010101010101010101072
:1037B00010101010100101010108010101010102A6
:1037C0001010101010101010101010101010100108
:1037D000010101040101010101021010101010107B
:1037E0001010101010101010100101010102010141
:1037F0000101010210101010101010101010101004
:10380000101010010101010101010101010210105C
:1038100010100810101010101010101010010101DD
:10382000010101010101010210101010041010101B
:10383000101010101010100101010101010101010F
:1038400001021010101002101010101010101010A3
:10385000100101010101010101010102101010100C
:1038600001101010101010101010100101010101B2
:1038700001010101010210101010001010101011B0
:1038800010101010100101010101010101010102DC
:103890001010101000101010101010101010110146
:1038A00001010101010101010102101010080010C5
:1038B0001010101010101010110101010101010170
:1038C000010101021010100400101010101010104F
:1038D000101011010101010101010101010210108B
:1038E0001002001010101010101010101101010122
:1038F000010101010101010210101001001010105E
:10390000101010101010110101010101010101013D
:1039100001021010100000101010111010101010E3
:10392000110101010101010101010102101010004A
:1039300000101010101010101011110101010101E0
:1039400001010101010210100800001010101010F8
:103950001010101111010101010101010101010209
:103960001010040000101010101010101011110190
:10397000010101010101010101021010020000100A
:10398000101010101010101111010101010101019E
:103990000101010210100100001010101010101091
:1039A00010111101010101010101010101021010B9
:1039B0000000001010111010101010111101010161
:1039C000010101010101010210100000001010109E
:1039D000101010101111110101010101010101016B
:1039E000010210080000001010101010101011112A
:1039F0001101010101010101010101021004000096
:103A0000001010101010101011111101010101010E
:103A1000010101010102100200000010101010103D
:103A20001010111111010101010101010101010237
:103A300010010000001010101010101011111101D1
:103A4000010101010101010101021000000000104B
:103A500011101010101011111101010101010101CB
:103A600001010102100000000010101010101011D0
:103A700011111101010101010101010101020800FF
:103A8000000000101010101010111111110101018F
:103A900001010101010101020400000000101010E9
:103AA0001010101111111101010101010101010199
:103AB000010202000000001010101010101111116E
:103AC00011010101010101010101010201000000D8
:103AD000001010101010101111111101010101013D
:103AE000010101010102000000000011101010107E
:103AF0001011111111010101010101010101010266
:103B0000000000000010101010101111111111010F
:103B1000010101010101010101021000000000008A
:103B200010101010111111111101010101010101F9
:103B3000010101021000000000101010101001110E
:103B40001111110101010101010101010102101016
:103B500000000010001010100111111111010101DD
:103B600001010101010101021010000000101010FC
:103B700010100101111111010101010101010101E7
:103B8000010210101000001010001010010111119E
:103B900011010101010101010101010210101000D8
:103BA000001010101010010101111101010101019B
:103BB000010101010102101010100010101000107E
:103BC00001010111110101010101010101010102C4
:103BD000101010100010101010100101010111013F
:103BE000010101010101010101021010101010106A
:103BF0001010100001010101110101010101010179
:103C0000010101021010101010101010101001010D
:103C10000101010101010101010101010102101075
:103C2000101008101010100801010101010101011C
:103C30000101010101010102081010100808101013
:103C4000100801010101010101010101010101014E
:103C500001021800100018180010001801010101DD
:103C60000101010101010101010101020C00080033
:103C70000C0C0008000C010101010101010101010E
:103C8000010101010102060004000606000400060D
:103C90000101010101010101010101010101010213
:103CA00003000400030300040003010101010101FA
:103CB00001010101010101010102020104010202ED
:103CC00001040102010101010101010101010101E0
:103CD00001010102020102010202010201020101CD
:103CE00001010101010101010101010101020101C3
:103CF00002010101010201010101010101010101B2
:103D0000010101010101010202020202020202029A
:103D10000202020202020202020202020202020283
:103D20000202030303030303030303030303030365
:103D30000303030303030303030303020707070744
:103D40000707070707070707070707070707070703
:103D50000707070707020F0F0F0F0F0F0F0F0F0FA8
:103D60000F0F0F0F0F0F0F0F0F0F0F0F0F0F0F0270
:103D70001F1F1F1F1F1F1F1F1F1F1F1F1F1F1F1F53
:103D80001F1F1F1F1F1F1F1F1F021E1E1E1E1E1E66
:103D90001E1E1E1E1E1E1E1E1E1E1E1E1E1E1E1E43
:103DA0001E1E1E021C1C1C1C1C1C1C1C1C1C1C1C67
:103DB0001C1C1C1C1C1C1C1C1C1C1C1C1C02181865
:103DC0001818181818181818181818181818181873
:103DD00018181818181818021010101010101010B9
:103DE00010101010101010101010101010101010D3
:103DF00010020000000000000000000000000000B1
:103E000000000000000000000000000200000000B0
:103E100000000000000000000000000000000000A2
:103E20000000000000020000000000000000000090
:103E30000000000000000000000000000000000280
:103E40000000000000000000000000000000000072
:103E50000000000000000000100200000000000050
:103E60000000000000000000000000000000000052
:103E70000010180200000000000000000000000018
:103E80000000000000000000000010101C020000F4
:103E90000000000000000000000000000000000022
:103EA0000000001010101E020000000000000000C2
:103EB00000000000000000000000000010101010C2
:103EC0001F020000000000000000000000000000D1
:103ED000000000000000181010111F020000000078
:103EE00000000000000000000000000000000000D2
:103EF0001C1011111F020000000000000000000053
:103F0000000000000000000000001E1111111F023F
:103F100000000000000000000000000000000000A1
:103F2000000000001F1111111F020000000000001E
:103F300000000000000000000000000000101F1141
:103F400011111F020000000000000000000000002E
:103F500000000000000010181F1111111F020000C6
:103F60000000000000000000000000000000001041
:103F7000101C1F1111111F020000000000000000A2
:103F800000000000000000001010101E1F11111191
:103F90001F02000000000000000000000000000000
:103FA00000101010101F1F1111111F02000000003F
:103FB0000000000000000000000000181010111F99
:103FC0001F1111111F02000000000000000000007E
:103FD00000000000001C1011111F1F1111111F0201
:103FE0000000000000000000000000000000001EB3
:103FF0001111111F1F1111111F02000000000000FC
:104000000000000000000000001F1111111F1F110F
:1040100011111F020000000000000000000000005D
:104020000000101F1111111F1F1111111F0200009C
:10403000000000000000000000000010181F111117
:10404000111F1F1111111F020000000000000000CD
:104050000000000010101C1F1111111F1F11111161
:104060001F020000000000000000000000101010FF
:104070001E1F1111111F1F1111111F02000000003E
:10408000000000000000101010101F1F1111111F60
:104090001F1111111F0200000000000000000000AD
:1040A000181010111F1F1111111F1F1111111F02C4
:1040B000000000000000000000001C1011111F1F74
:1040C0001111111F1F1111111F020000000000002B
:1040D000000000001E1111111F1F1111111F1F11CF
:1040E00011111F02000000000000000000001F115D
:1040F00011111F1F1111111F1F1111111F0200009B
:1041000000000000000000101F1111111F1F1111ED
:10411000111F1F1111111F020000000000000000FC
:1041200010181F1111111F1F1111111F1F11111133
:104130001F020000000000000010101C1F111111D0
:104140001F1F1111111F1F1111111F02000000006C
:1041500000001010101E1F1111111F1F1111111F2F
:104160001F1111111F020000000000101010101F7D
:104170001F1111111F1F1111111F1F1111111F02EA
:104180000000000000181010111F1F1111111F1F37
:104190001111111F1F1111111F0200000000001C3E
:1041A0001011111F1F1111111F1F1111111F1F11AC
:1041B00011111F0200000000001E1111111F1F111C
:1041C00011111F1F1111111F1F1111111F020000CA
:1041D0000000001F1111111F1F1111111F1F1111BC
:1041E000111F1F1111111F0200000000101F1111DB
:1041F000111F1F1111111F1F1111111F1F1111115B
:104200001F0200000010181F1111111F1F111111A2
:104210001F1F1111111F1F1111111F02000010107B
:104220001C1F1111111F1F1111111F1F1111111F1F
:104230001F1111111F02001010101E1F1111111F4C
:104240001F1111111F1F1111111F1F1111111F0219
:10425000101010101F1F1111111F1F1111111F1FFE
:104260001111111F1F1111111F02181010111F1F02
:104270001111111F1F1111111F1F1111111F1F11DA
:1042800011111F021C1011111F1F1111111F1F11DD
:1042900011111F1F1111111F1F1111111F021E11CA
:1042A00011111F1F1111111F1F1111111F1F1111AA
:1042B000111F1F1111111F021F1111111F1F1111A9
:1042C000111F1F1111111F1F1111111F1F1111118A
:1042D0001F021F1111111F1F1111111F1F11111189
:1042E0001F1F1111111F1F1111111F021F11111179
:1042F0000F1F1111111F1F1111111F1F1111111F5C
:104300001F1111111F021F111101071F1111111F80
:104310001F1111111F1F1111111F1F1111111F0248
:104320001F110101031F1111111F1F1111111F1F57
:104330001111111F1F1111111F021F010101011F76
:104340001111111F1F1111111F1F1111111F1F1109
:1043500011111F020F010101001F1111111F1F1167
:1043600011111F1F1111111F1F1111111F02070120
:104370000100001F1111111F1F1111111F1F111119
:10438000111F1F1111111F0203010000001F111145
:10439000111F1F1111111F1F1111111F1F111111B9
:1043A0001F0201000000001F1111111F1F11111128
:1043B0001F1F1111111F1F1111111F0200000000FA
:1043C000001F1111111F1F1111111F1F1111111F9A
:1043D0001F1111111F0200000000001F1111110F09
:1043E0001F1111111F1F1111111F1F1111111F0278
:1043F00000000000001F111101071F1111111F1FE4
:104400001111111F1F1111111F0200000000001FC8
:10441000110101031F1111111F1F1111111F1F1174
:1044200011111F0200000000001F010101011F11F6
:1044300011111F1F1111111F1F1111111F02000057
:104440000000000F010101001F1111111F1F1111A8
:10445000111F1F1111111F020000000000070101B0
:1044600000001F1111111F1F1111111F1F11111118
:104470001F02000000000003010000001F111111C5
:104480001F1F1111111F1F1111111F020000000029
:104490000001000000001F1111111F1F1111111F39
:1044A0001F1111111F020000000000000000000099
:1044B0001F1111111F1F1111111F1F1111111F02A7
:1044C000000000000000000000001F1111110F1F6C
:1044D0001111111F1F1111111F0200000000000017
:1044E000000000001F111101071F1111111F1F11E2
:1044F00011111F02000000000000000000001F1149
:104500000101031F1111111F1F1111111F020000C2
:1045100000000000000000001F010101011F111137
:10452000111F1F1111111F020000000000000000E8
:1045300000000F010101001F1111111F1F111111A6
:104540001F02000000000000000000000701010041
:10455000001F1111111F1F1111111F020000000077
:1045600000000000000003010000001F1111111FD6
:104570001F1111111F0200000000000000000000C8
:1045800001000000001F1111111F1F1111111F0246
:104590000000000000000000000000000000001FFC
:1045A0001111111F1F1111111F0200000000000046
:1045B0000000000000000000001F1111110F1F116A
:1045C00011111F02000000000000000000000000A8
:1045D0000000001F111101071F1111111F0200001F
:1045E000000000000000000000000000001F11019A
:1045F00001031F1111111F02000000000000000044
:10460000000000000000001F010101011F11111135
:104610001F02000000000000000000000000000079
:10462000000F010101001F1111111F020000000005
:104630000000000000000000000000070101000071
:104640001F1111111F0200000000000000000000F7
:10465000000000000003010000001F1111111F02E3
:104660000000000000000000000000000000000149
:10467000000000001F1111111F02000000000000C7
:1046800000000000000000000000000000001F11FA
:1046900011111F02000000000000000000000000D7
:1046A00000000000000000001F1111110F020000A7
:1046B00000000000000000000000000000000000FA
:1046C00000001F111101070200000000000000009F
:1046D0000000000000000000000000001F110101A8
:1046E00003020000000000000000000000000000C5
:1046F0000000000000001F01010101020000000095
:1047000000000000000000000000000000000000A9
:104710000F01010100020000000000000000000085
:10472000000000000000000000000701010000027E
:104730000000000000000000000000000000000079
:104740000000000003010000000200000000000063
:104750000000000000000000000000000000010058
:104760000000000200000000000000000000000047
:10477000000000000000000000000000000A00002F
:1047800000000E00000011000000110000001100E8
:1047900000000E00000000070001010100020000FF
:1047A00000020400000004080000000800101010BF
:1047B00000070E00000000001100000000001100C2
:1047C000000000001100000000000E070010101093
:1047D00000080000000804000000040200000002BD
:1047E000000101010007000000000E0000001100A0
:1047F000000011000000110000000E000000000683
:104800000001010100020000000204000000040891
:10481000000000080010101000060E00000000004C
:104820001100000000001100000000001100000055
:1048300000000E0600101010000800000008040020
:104840000000040200000002000101010006000057
:1048500000000E0000001100000011000000110017
:1048600000000E0000000005000101010002000030
:1048700000020400000004080000000800101010EE
:1048800000050E00000000001100000000001100F3
:10489000000000001100000000000E0500101010C4
:1048A00000080000000804000000040200000002EC
:1048B000000101010005000000000E0000001100D1
:1048C000000011000000110000000E0000000004B4
:1048D00000010101000200000002040000000408C1
:1048E000000000080010101000040E00000000007E
:1048F0001100000000001100000000001100000085
:1049000000000E0400101010000800000008040051
:104910000000040200000002000101010004000088
:1049200000000E0000001100000011000000110046
:1049300000000E0000000003000101010002000061
:10494000000204000000040800000008001010101D
:1049500000030E0000000000110000000000110024
:10496000000000001100000000000E0300101010F5
:10497000000800000008040000000402000000021B
:10498000000101010003000000000E000000110002
:10499000000011000000110000000E0000000002E5
:1049A00000010101000200000002040000000408F0
:1049B000000000080010101000020E0000000000AF
:1049C00011000000000011000000000011000000B4
:1049D00000000E0200101010000800000008040083
:1049E00000000402000000020001010100020000BA
:1049F00000000E0000001100000011000000110076
:104A000000000E0000000002000101010002000091
:104A1000000204000000040800000008001010104C
:104A200000020E0000000000110000000000110054
:104A3000000000001100000000000E020010101025
:104A4000000800000008040000000402000000024A
:104A5000000101010002000000000E000000110032
:104A6000000011000000110000000E000000000214
:104A7000000101010002000000020400000004081F
:104A8000000000080010101000020E0000000000DE
:104A900011000000000011000000000011000000E3
:104AA00000000E02001010100008000000080400B2
:104AB00000000402000000020001010100020000E9
:104AC00000000E00000011000000110000001100A5
:104AD00000000E00000000020001010100020000C1
:104AE000000204000000040800000008001010107C
:104AF00000020E0000000000110000000000110084
:104B0000000000001100000000000E020010101054
:104B10000008000000080400000004020000000279
:104B20000001010100020000000000000000000080
:104B3000000000000000000000000E1111110E0A1C
:104B40000000000000000000000000000000000065
:104B5000000000000E1111110E0A000000000000FC
:104B600000000000000000000000000000000E1126
:104B700011110E0200000000000000000000000003
:104B8000000000000000000000000000000A00001B
:104B900000000000001F0000001F001F001F000099
:104BA000001F1F0000001F0A000000000000001F7F
:104BB0000000001F001F001F0000001F0000000079
:104BC000000A000000000000000000001F1F1F1F5F
:104BD0001F000000000000000000000A00000000AC
:104BE000001F0000001F001F001F0000001F00002A
:104BF00000000000000A1F0000001F1F0000001F2F
:104C0000001F001F0000001F000000000000000A3D
:104C100000000000001F0000001F001F001F000018
:104C2000001F000000000000000A0000000000005B
:104C3000000000001F1F1F1F1F00000000000000D9
:104C40000000000A000000000000001F0000001F1C
:104C5000001F001F0000001F00000000000A0000ED
:104C600000000000001F0000001F001F001F0000C8
:104C7000001F1F0000001F07000000000000001FB1
:104C80000000001F001F001F0000001F00000000A8
:104C90000007000000000000000000001F1F1F1F91
:104CA0001F000000000000000000000700000000DE
:104CB000001F0000001F001F001F0000001F000059
:104CC0000000000000071F0000001F1F0000001F61
:104CD000001F001F0000001F000000000000000770
:104CE00000000000001F0000001F001F001F000048
:104CF000001F00000000000000070000000000008E
:104D0000000000001F1F1F1F1F0000000000000008
:104D100000000007000000000000001F0000001F4E
:104D2000001F001F0000001F00000000000700001F
:104D30000000000000000000000000000000000073
:104D4000000000000000000700000000100000004C
:104D50000010000000001000000000100000000023
:104D600010050000001018000000101800000010CE
:104D7000180000001018000000101805000010189E
:104D80001C000010181C000010181C000010181C3B
:104D9000000010181C050010181C1E0010181C1E06
:104DA0000010181C1E0010181C1E0010181C1E05D8
:104DB00010181C1E1F10181C1E1F10181C1E1F1060
:104DC000181C1E1F10181C1E1F05181C1E1F1F1844
:104DD0001C1E1F1F181C1E1F1F181C1E1F1F181C07
:104DE0001E1F1F051C1E1F1F1F1C1E1F1F1F1C1EFA
:104DF0001F1F1F1C1E1F1F1F1C1E1F1F1F051E1FE6
:104E00001F1F1F1E1F1F1F1F1E1F1F1F1F1E1F1FB5
:104E10001F1F1E1F1F1F1F051F1F1F1F1F1F1F1FBD
:104E20001F1F1F1F1F1F1F1F1F1F1F1F1F1F1F1F92
:104E30001F051F1F1F1F0F1F1F1F1F0F1F1F1F1FBC
:104E40000F1F1F1F1F0F1F1F1F1F0F051F1F1F0FCC
:104E5000071F1F1F0F071F1F1F0F071F1F1F0F07F2
:104E60001F1F1F0F07051F1F0F07031F1F0F07031C
:104E70001F1F0F07031F1F0F07031F1F0F07030528
:104E80001F0F0703011F0F0703011F0F0703011F58
:104E90000F0703011F0F070301050F070301000F91
:104EA000070301000F070301000F070301000F07AD
:104EB00003010005070301000007030100000703C9
:104EC00001000007030100000703010000050301C2
:104ED00000000003010000000301000000030100C6
:104EE00000000301000000050100000000010000B7
:104EF00000000100000000010000000001000000AF
:104F0000000500000000000000000000000000009C
:104F1000000000000000000000000005100000007C
:104F20000010000000001000000000100000000051
:104F3000100000000005181000000018100000000C
:104F400018100000001810000000181000000005E4
:104F50001C181000001C181000001C181000001C69
:104F6000181000001C18100000051E1C1810001E50
:104F70001C1810001E1C1810001E1C1810001E1CEF
:104F8000181000051F1E1C18101F1E1C18101F1EB5
:104F90001C18101F1E1C18101F1E1C1810051F1F88
:104FA0001E1C181F1F1E1C181F1F1E1C181F1F1E33
:104FB0001C181F1F1E1C18051F1F1F1E1C1F1F1F34
:104FC0001E1C1F1F1F1E1C1F1F1F1E1C1F1F1F1EFE
:104FD0001C051F1F1F1F1E1F1F1F1F1E1F1F1F1F00
:104FE0001E1F1F1F1F1E1F1F1F1F1E051F1F1F1FEE
:104FF0001F1F1F1F1F1F1F1F1F1F1F1F1F1F1F1FC1
:105000001F1F1F1F1F050F1F1F1F1F0F1F1F1F1FEA
:105010000F1F1F1F1F0F1F1F1F1F0F1F1F1F1F05EA
:10502000070F1F1F1F070F1F1F1F070F1F1F1F0720
:105030000F1F1F1F070F1F1F1F0503070F1F1F0332
:10504000070F1F1F03070F1F1F03070F1F1F030754
:105050000F1F1F050103070F1F0103070F1F010388
:10506000070F1F0103070F1F0103070F1F05000193
:1050700003070F000103070F000103070F000103DF
:10508000070F000103070F050000010307000001DF
:1050900003070000010307000001030700000103EC
:1050A00007050000000103000000010300000001EB
:1050B00003000000010300000001030500000000E0
:1050C00001000000000100000000010000000001DC
:1050D00000000000010500000000000000000000CA
:1050E00000000000000000000000000000000005BB
:1050F00001000000000100000000010000000001AC
:105100000000000001000000000503010000000392
:105110000100000003010000000301000000030182
:10512000000000050703010000070301000007035A
:1051300001000007030100000703010000050F073D
:105140000301000F070301000F070301000F07030E
:1051500001000F07030100051F0F0703011F0F07C1
:1051600003011F0F0703011F0F0703011F0F070391
:1051700001051F1F0F07031F1F0F07031F1F0F0727
:10518000031F1F0F07031F1F0F0703051F1F1F0FFD
:10519000071F1F1F0F071F1F1F0F071F1F1F0F07AF
:1051A0001F1F1F0F07051F1F1F1F0F1F1F1F1F0F71
:1051B0001F1F1F1F0F1F1F1F1F0F1F1F1F1F0F0549
:1051C0001F1F1F1F1F1F1F1F1F1F1F1F1F1F1F1FEF
:1051D0001F1F1F1F1F1F1F1F1F051E1F1F1F1F1EFB
:1051E0001F1F1F1F1E1F1F1F1F1E1F1F1F1F1E1FD2
:1051F0001F1F1F051C1E1F1F1F1C1E1F1F1F1C1EE5
:105200001F1F1F1C1E1F1F1F1C1E1F1F1F05181CDA
:105210001E1F1F181C1E1F1F181C1E1F1F181C1EC0
:105220001F1F181C1E1F1F0510181C1E1F10181CE6
:105230001E1F10181C1E1F10181C1E1F10181C1ECD
:105240001F050010181C1E0010181C1E0010181C32
:105250001E0010181C1E0010181C1E05000010183F
:105260001C000010181C000010181C000010181C56
:10527000000010181C050000001018000000101895
:1052800000000010180000001018000000101805A1
:1052900000000000100000000010000000001000DE
:1052A00000000010000000001005000000000000D9
:1052B00000000000000000000000000000000000EE
:1052C00000000005000000000100000000010000D7
:1052D00000000100000000010000000001050000C6
:1052E00000010300000001030000000103000000B2
:1052F0000103000000010305000001030700000195
:105300000307000001030700000103070000010379
:105310000705000103070F000103070F0001030742
:105320000F000103070F000103070F050103070F1B
:105330001F0103070F1F0103070F1F0103070F1FA3
:105340000103070F1F0503070F1F1F03070F1F1F71
:1053500003070F1F1F03070F1F1F03070F1F1F0543
:10536000070F1F1F1F070F1F1F1F070F1F1F1F07DD
:105370000F1F1F1F070F1F1F1F050F1F1F1F1F0FAF
:105380001F1F1F1F0F1F1F1F1F0F1F1F1F1F0F1F5D
:105390001F1F1F051F1F1F1F1F1F1F1F1F1F1F1F37
:1053A0001F1F1F1F1F1F1F1F1F1F1F1F1F051F1F27
:1053B0001F1F1E1F1F1F1F1E1F1F1F1F1E1F1F1F00
:1053C0001F1E1F1F1F1F1E051F1F1F1E1C1F1F1F0D
:1053D0001E1C1F1F1F1E1C1F1F1F1E1C1F1F1F1EEA
:1053E0001C051F1F1E1C181F1F1E1C181F1F1E1C04
:1053F000181F1F1E1C181F1F1E1C18051F1E1C18FF
:10540000101F1E1C18101F1E1C18101F1E1C181009
:105410001F1E1C1810051E1C1810001E1C18100042
:105420001E1C1810001E1C1810001E1C1810000551
:105430001C181000001C181000001C181000001C84
:10544000181000001C1810000005181000000018AB
:1054500010000000181000000018100000001810C4
:105460000000000510000000001000000000100007
:105470000000001000000000100000000005000007
:10548000000000000000000000000000000000001C
:1054900000000000000000051010101010000000B7
:1054A00000000000000000000000000000000000FC
:1054B000000518181818181010101010000000001F
:1054C0000000000000000000000000051C1C1C1C67
:1054D0001C181818181810101010100000000000E8
:1054E0000000000000051E1E1E1E1E1C1C1C1C1C95
:1054F00018181818181010101010000000000005DF
:105500001F1F1F1F1F1E1E1E1E1E1C1C1C1C1C18C6
:10551000181818181010101010051F1F1F1F1F1F1C
:105520001F1F1F1F1E1E1E1E1E1C1C1C1C1C1818AD
:10553000181818051F1F1F1F1F1F1F1F1F1F1F1FAA
:105540001F1F1F1E1E1E1E1E1C1C1C1C1C051F1F99
:105550001F1F1F1F1F1F1F1F1F1F1F1F1F1F1F1F5B
:105560001F1F1E1E1E1E1E051F1F1F1F1F1F1F1F6A
:105570001F1F1F1F1F1F1F1F1F1F1F1F1F1F1F1F3B
:105580001F050F0F0F0F0F1F1F1F1F1F1F1F1F1F95
:105590001F1F1F1F1F1F1F1F1F1F1F050707070795
:1055A000070F0F0F0F0F1F1F1F1F1F1F1F1F1F1F73
:1055B0001F1F1F1F1F050303030303070707070719
:1055C0000F0F0F0F0F1F1F1F1F1F1F1F1F1F1F0555
:1055D0000101010101030303030307070707070F85
:1055E0000F0F0F0F1F1F1F1F1F05000000000001DE
:1055F00001010101030303030307070707070F0F57
:105600000F0F0F0500000000000000000000010166
:105610000101010303030303070707070705000050
:105620000000000000000000000000000001010177
:105630000101030303030305000000000000000054
:105640000000000000000000000000000101010156
:105650000105000000000000000000000000000044
:105660000000000000000000000000050000000035
:10567000000000000000000000000000000000002A
:105680000000000000050000000000000000000015
:105690000000000000000000000000000000000505
:1056A00010000000010010000100000011000000C7
:1056B0000100100001000000100A040000000408AE
:1056C00000000002100000000100100001000000B6
:1056D0001100000A01000000100200000008040090
:1056E000000004080000000210000000010A000091
:1056F0001100000001001000010000001002000075
:10570000000804000000040A10000000010010005E
:105710000100000011000000010010000100000065
:10572000100A04000000040800000002100000003D
:1057300001001000010000001100000A010000003B
:10574000100200000008040000000408000000022D
:1057500010000000010A000011000000010010000C
:105760000100000010020000000804000000040A0C
:10577000040A150A040201001008010000001000CC
:1057800000000000000000000005040A150A0402E1
:1057900001001008010000000002010000000000EC
:1057A00000000005040A150A0402010000000100BF
:1057B0000000000201000000040201000005040ACC
:1057C00005020002010000000100000000020100CB
:1057D0000000040A050200050402010000020100A5
:1057E000000001000000000201000000040A150A88
:1057F000040500000000000201000000010000009C
:10580000000201001008040A150A04050000000047
:10581000000000000000010000001002010010085C
:10582000040A150A0405000000000000000010082A
:1058300000000000100201001008040A150A040507
:105840000000100804000000100800000000100014
:1058500000001008040A150A04050008140A0400D0
:1058600000001008000000001000000010080008F0
:10587000140A0405040A150A0400000010080000B8
:105880000000100000001008000010080405040AC1
:10589000150A0402010010080000000010000000BA
:1058A0001008000000000005040A150A04020100A7
:1058B00010080100000010000000000000000000BF
:1058C0000005040A150A0402010010080100000086
:1058D000000201000000000000000005040A150A93
:1058E00004020100000001000000000201000000AD
:1058F000040201000005040A050200020100000084
:1059000001000000000201000000040A0502000579
:10591000040201000002010000000100000000027A
:1059200001000000040A150A04050000000000023E
:105930000100000001000000000201001008040A3C
:10594000150A04050000000000000000000001002E
:105950000000100201001008040A150A04050000E6
:10596000000000000000100800000000100201000C
:105970001008040A150A04050000100804000000BD
:10598000100800000000100000001008040A150AAA
:1059900004050008140A04000000100800000000BC
:1059A0001000000010080008140A0405040A150A73
:1059B00004000000100800000000100000001008A3
:1059C000000010080405040A150A0402010010086A
:1059D000000000001000000010080000000000059A
:1059E000040A150A0402010010080100000010005A
:1059F00000000000000000000005040A150A04026F
:105A00000100100801000000000201000000000079
:105A100000000005040A150A04020100000001004C
:105A20000000000201000000040201000005040A59
:105A30000502000201000000010000000002010058
:105A40000000040A05020005040201000002010032
:105A5000000001000000000201000000040A150A15
:105A60000405000000000002010000000100000029
:105A7000000201001008040A150A040500000000D5
:105A800000000000000001000000100201001008EA
:105A9000040A150A040500000000000000001008B8
:105AA00000000000100201001008040A150A040595
:105AB00000001008040000001008000000001000A2
:105AC00000001008040A150A04050008140A04005E
:105AD000000010080000000010000000100800087E
:105AE000140A0405040A150A040000001008000046
:105AF0000000100000001008000010080405040A4F
:105B0000150A040201001008000000001000000047
:105B10001008000000000005000000000000000068
:105B20000000000000000000000000000000000075
:105B3000000A00000000000000000000000000005B
:105B400000000000000000000000000AFFFFFFFF4F
:105B5000FFFFFFFFFFFFFFFFFFFFFFFFFFFFFFFF55
:105B6000FFFFFFFFFFFFFFFFFFFFFFFFFFFFFFFF45
:105B7000FFFFFFFFFFFFFFFFFFFFFFFFFFFFFFFF35
:105B8000FFFFFFFFFFFFFFFFFFFFFFFFFFFFFFFF25
:107C00000C942A3E0C94473E0C94473E0C94473EFD
:107C10000C94473E0C94473E0C94473E0C94473ED0
:107C20000C94473E0C94473E0C94473E0C94473EC0
:107C30000C94473E0C94473E0C94473E0C94473EB0
:107C40000C94473E0C94473E0C94473E0C94473EA0
:107C50000C94473E11241FBECFE5D8E0DEBFCDBF58
:107C600010E0A0E6B0E0E4EBFEE702C005900D9264
:107C7000A236B107D9F710E0A2E6B0E001C01D922C
:107C8000A038B107E1F70E94333F0C94583F0C94A1
:107C9000003E0C94000008955F9BFECF8CB1E6E699
:107CA000F0E05F9BFECF8CB1819380E0E038F80775
:107CB000C1F75F9BFECF8CB10895FF920F931F9386
:107CC000CF93DF936091600070916100209162001A
:107CD00030916300A6E6B0E083E0F82E05E011E005
:107CE0002038310591F4FB01F0925700E89507B672
:107CF00000FCFDCFFB0100935700E89507B600FCA0
:107D0000FDCF60587F4F20E030E08C91F901E60F05
:107D1000F71F11965C91119740E0EA01C80FD11D41
:107D20000E0110935700E89511242E5F3F4F1296D5
:107D3000E0E0A038BE07A1F6709361006093600098
:107D40003093630020936200DF91CF911F910F91D8
:107D5000FF900895E0916000F091610085E08093CC
:107D60005700E89507B600FCFDCF0895E09160004C
:107D7000F091610083E080935700E89507B600FC1E
:107D8000FDCF08955F9BFECF3CB15F9BFECF2CB132
:107D9000922F80E0830F911D909365008093640083
:107DA000E0E8F3E121E00C0120935700E89511246D
:107DB00083E080935700E89507B600FCFDCFE0E82C
:107DC000F3E185E080935700E89507B600FCFDCF0E
:107DD00008950F931F93CF93DF930E94C23EC0E09C
:107DE000D0E004E01EE719C088B3802788BB5F9B02
:107DF000FECF8CB1E6E6F0E05F9BFECF8CB18193C5
:107E000080E0E038F807C1F75F9BFECF8CB10E949D
:107E10005D3E5D9BFECF1CB92196809164009091E0
:107E20006500C817D90700F3E0916000F091610088
:107E300083E080935700E89507B600FCFDCF85E00E
:107E400080935700E89507B600FCFDCF81E1809351
:107E50005700E8955D9BFECF83E48CB9DF91CF910D
:107E60001F910F9108951F930E944D3F84E087BB9F
:107E700014E5C2985F9BFECF8CB1823519F40C9447
:107E80000000F7CF8A3219F40E94E93EF2CF843520
:107E900081F75D9BFECF1CB9ECCF10BC8BE089B99C
:107EA00088E18AB986E880BD8CB15F99FDCF0895DD
:107EB000F894FFCF0014FFFFFFFFFFFFFFFFFFFF5E
:107EC000FFFFFFFFFFFFFFFFFFFFFFFFFFFFFFFFC2
:107ED000FFFFFFFFFFFFFFFFFFFFFFFFFFFFFFFFB2
:107EE000FFFFFFFFFFFFFFFFFFFFFFFFFFFFFFFFA2
:107EF000FFFFFFFFFFFFFFFFFFFFFFFFFFFFFFFF92
:107F0000FFFFFFFFFFFFFFFFFFFFFFFFFFFFFFFF81
:107F1000FFFFFFFFFFFFFFFFFFFFFFFFFFFFFFFF71
:107F2000FFFFFFFFFFFFFFFFFFFFFFFFFFFFFFFF61
:107F3000FFFFFFFFFFFFFFFFFFFFFFFFFFFFFFFF51
:107F4000FFFFFFFFFFFFFFFFFFFFFFFFFFFFFFFF41
:107F5000FFFFFFFFFFFFFFFFFFFFFFFFFFFFFFFF31
:107F6000FFFFFFFFFFFFFFFFFFFFFFFFFFFFFFFF21
:107F7000FFFFFFFFFFFFFFFFFFFFFFFFFFFFFFFF11
:107F8000FFFFFFFFFFFFFFFFFFFFFFFFFFFFFFFF01
:107F9000FFFFFFFFFFFFFFFFFFFFFFFFFFFFFFFFF1
:107FA000FFFFFFFFFFFFFFFFFFFFFFFFFFFFFFFFE1
:107FB000FFFFFFFFFFFFFFFFFFFFFFFFFFFFFFFFD1
:107FC000FFFFFFFFFFFFFFFFFFFFFFFFFFFFFFFFC1
:107FD000FFFFFFFFFFFFFFFFFFFFFFFFFFFFFFFFB1
:107FE000FFFFFFFFFFFFFFFFFFFFFFFFFFFFFFFFA1
:107FF000FFFFFFFFFFFFFFFFFFFFFFFFFFFFFFFF91
:00000001FF
